:1000000000308A0004280000FF238316900000308F
:100010008A005B2B820720342034203420342034A3
:10002000523461346C3465346E34743469347334EE
:1000300073346534753472345F34733465347234B8
:1000400076346F345F3431343234463436343734B6
:1000500035345F345634303432342D343034353422
:1000600000340034003400340034003400343330C1
:100070008400000803194B280130A100A001A00B47
:100080003F28A10B3E284A30A000A00B45280000C5
:100090000000800B3C28882B0C30A1001F08C339BE
:1000A00021049F000330A000A00B54289F149F1828
:1000B00057281E08A700A70E0F30A7050430A1007F
:1000C0001F08C33921049F000330A000A00B66283D
:1000D0009F149F1869281E08A900A90E0F30A905B2
:1000E00000342510A601A801AA08031978280030B9
:1000F0004C20892B90018F018E010C1085309000CF
:10010000B401B5013310003033180130003A031D3B
:10011000CE28003085190130013C031D9C28340B8A
:100120009428B40A0F08B6003408033C031D9B282A
:10013000B40A0F08B800A828B408031DA12801308C
:10014000B4003408023C031DA828B40A0F08B70005
:10015000003005190130013C031DBB28350BB328C5
:10016000B50A0F08B9003508033C031DBA28B50AC3
:100170000F08BB00C728B508031DC0280130B50013
:100180003508023C031DC728B50A0F08BA00003025
:100190000C180130013C0319331483289001B3106B
:1001A00033113408043C031DE128B3143608380227
:1001B000BC003C08393C0318E0283C08643C031CA4
:1001C000B310AA013508043C031DF2283315390881
:1001D0003B02BC003C08393C0318F1283C08643C55
:1001E000031C3311B31C1629331D16293908360296
:1001F0000318082936083902BD00390838023D02C3
:10020000031805290330AA0007290430AA0015297C
:1002100039083602BD0036083B023D020318132997
:100220000430AA0015290330AA001E29B31C1A297C
:100230000130AA00331D1E290230AA008A2B90012A
:100240008F018E010C10003085190130003A03191E
:10025000232985309000003085190130013C0319B5
:100260002B2990010F08A3000E08A0000F082302FD
:10027000031D32292008AD002308AE0025100030F0
:100280000C180130013C031925142E08033C031CF3
:100290004F29031D4E292D081F3C031825142E0835
:1002A000083C03185A29FF3A031D59292D08C43C5C
:1002B000031C25140034B601B50135083F3C031C6E
:1002C0006B292708260203186729A60A6929A601AF
:1002D000B60AB50A5D293608AB070318AC0A2E0822
:1002E0002C02031C7E29031D79292B082D020318DB
:1002F0007E292E08AC002D08AB00A6010034B60103
:10030000B50135083F3C031C8F2927082602031836
:100310008B29A60A8D29A601B60AB50A81293608B5
:10032000AB020030031C0130AC022C082E02031C6F
:10033000A429031D9F292D082B020318A4292E0888
:10034000AC002D08AB00A60100342B08003CB50022
:10035000B6012C08031C2C0FB6020130B700003088
:10036000031C0130B702B8010030031C0130B80291
:1003700036088F0035088E000C10851685309000E9
:1003800000300C180130003A0319C02985120034DE
:1003900025101F21003025180130003A031D022AC4
:1003A0002D082B02B3002C08B4002E08031C2E0FBE
:1003B000B402B408031DE0293308073C0318012ADE
:1003C0003408FE3C0318EB29FF3A031D012A3308C9
:1003D000F83C031C012A2C082E02031CF729031DDC
:1003E000F5292D082B020318F7295B21012A2E0875
:1003F0002C02031C012A031D002A2B082D02031CBA
:100400007F21A521A32B90018F018E010C100030BC
:1004100005190130003A0319072A85309000003091
:1004200005190130013C03190F2A90010F08A300A0
:100430000E08A0000F082302031D162A2008B10091
:100440002308B20000300C180130013C03192514B8
:100450003208033C031C322A031D312A31081F3C99
:10046000031825143208083C03183D2AFF3A031DDF
:100470003C2A3108C43C031C25140034B601B501E4
:1004800035083F3C031C4E2A2908280203184A2A33
:10049000A80A4C2AA801B60AB50A402A3608AF07AE
:1004A0000318B00A32083002031C612A031D5C2ABB
:1004B0002F0831020318612A3208B0003108AF005A
:1004C000A8010034B601B50135083F3C031C722A6F
:1004D0002908280203186E2AA80A702AA801B60A59
:1004E000B50A642A3608AF020030031C0130B0029E
:1004F00030083202031C872A031D822A31082F028A
:100500000318872A3208B0003108AF00A801003470
:100510002F08003CB500B6013008031C300FB602AE
:100520000130B7000030031C0130B702B8010030C1
:10053000031C0130B80236088F0035088E000C10FD
:1005400005148530900000300C180130003A031972
:10055000A32A05100034251003220030251801308D
:10056000003A031DE52A31082F02B3003008B40019
:100570003208031C320FB402B408031DC32A330827
:10058000073C0318E42A3408FE3C0318CE2AFF3A3D
:10059000031DE42A3308F83C031CE42A3008320225
:1005A000031CDA2A031DD82A31082F020318DA2A7D
:1005B0003E22E42A32083002031CE42A031DE32A07
:1005C0002F083102031C62228822BF2B25102A0823
:1005D000033C031DEE2A1F210322F02A03221F21C0
:1005E000003025180130003A031D5A2B2D082B022C
:1005F000B3002C08B4002E08031C2E0FB402B4085C
:10060000031D062B3308073C0318272B3408FE3C38
:100610000318112BFF3A031D272B3308F83C031C4A
:10062000272B2C082E02031C1D2B031D1B2B2D0812
:100630002B0203181D2B5B21272B2E082C02031CD9
:10064000272B031D262B2B082D02031C7F2131088D
:100650002F02B3003008B4003208031C320FB4027A
:10066000B408031D372B3308073C0318582B3408F4
:10067000FE3C0318422BFF3A031D582B3308F83C6D
:10068000031C582B30083202031C4E2B031D4C2B2D
:1006900031082F0203184E2B3E22582B320830020D
:1006A000031C582B031D572B2F083102031C6222F9
:1006B000A5218822E42B84011F30830583161F089F
:1006C000F0399F0083121F1307309F0007309900F5
:1006D0008316050803308312A000A00B6D2B1908A8
:1006E0008C1185013F30650083161F08F0390A38E8
:1006F0009F0083121F1383161F080F3930389F0085
:1007000083121F080C3901389F00C830B300372806
:1007100071287A2825102A0BA52B00308519013065
:10072000013C03198D2B1F21003025180130013C9D
:10073000031D9C2B8A0100281F3065002E08AC0089
:100740002D08AB00C8294C20A22B2A08023C031D0F
:10075000C12B003005190130013C0319A92B0322DC
:10076000003025180130013C031DB82B8A010028F8
:100770003E3065003208B0003108AF00AB2A4C2093
:10078000BE2B2A08033C0319C92B2A08043C031D6D
:10079000E62B003085190130013C0319C92B1F21BC
:1007A0000322003025180130013C031DD92B8A019A
:1007B00000281E3065002E08AC002D08AB00320862
:1007C000B0003108AF00E62A4C20E32B8A01002854
:0207D0006300C4
:02400E00C439B3
:00000001FF
